:1000000025C047C046C045C044C043C042C041C0EF
:1000100040C03FC03EC03DC03CC03BC03AC08B99D1
:10002000A2ABB0B4B9BEC2FF03146EE6FFFFFFFF80
:10003000000000000007385A89FF01020305060886
:1000400009000204070900F3F4EE090011241FBEA1
:10005000CFE5D1E0DEBFCDBF20E0A0E6B0E001C03B
:100060001D92A138B207E1F7E1E6F0E0128281E0EB
:100070008683ABE6B0E09EEF15969C9315979DEFB7
:1000800017969C93808788E58187612C712C92D08C
:100090002DC2B6CF815090E0FC01E85DFF4FE491A6
:1000A000E9BDFC01EF5CFF4F849188BD089520ED10
:1000B00037E0019720F0F9013197F1F7FACF089571
:1000C00088EE93E0F4CF81EA87B986EC86B9369A58
:1000D0000895369A3699FECF85B10895CF93C72DEE
:1000E00081E0870D8F73782E662D90E0F1D16FEF50
:1000F0008C2F90E0CF91ECC1FF920F931F93CF9381
:10010000DF93F82E0AE610E0C6E7D0E081E0F812AF
:1001100005C0F8016081CE01DBD104C0CE01D0D191
:10012000F8018083015011092196CF37D10571F76D
:10013000DF91CF911F910F91FF900895CFDF81E064
:10014000DBCF811103C019BC18BC0895A3CF0F9356
:100150001F93CF93C82F8B01CC2361F082E09ADFED
:10016000C801A5DF19BC18BCC801A1DFC8019FDF09
:10017000C150F2CFCF911F910F9108951F93CF934C
:10018000DF938FEA87B986EC86B910E1C0E0D0E052
:1001900085E090E08CDF9DDFC80FD11D1150C1F7C5
:1001A000CE0124E0969587952A95E1F7DF91CF91CE
:1001B0001F91089583EA87B986EC86B93699FECFF8
:1001C000369A86B1D82FD07486FDFBCF15B18FE358
:1001D00084BBBB9AC39AB99AB89A81E08ABD83BF9F
:1001E0008AB580628ABD8AB580688ABD97B328B314
:1001F000892F90E0809590958B7F822B88BB712C06
:10020000872D90E05DD1682E8F3F09F056C1872D74
:1002100091E0970D792E803498F390DF209169005A
:100220002F5F4AE350E0222391F0CA010196FC01BE
:100230003197E491AD2FB0E0AD58BF4FEC93EE2372
:1002400019F0D82FD41BF2CF2150AC01ECCFD093B2
:10025000600084E08D0F982F9150E92FED1BF0E0A6
:10026000E95BFF4FE491A92FB0E0AD58BF4FEC938D
:100270009D13F2CFE82FF0E0EE58FF4F91E0309160
:1002800073002081321390E0891B982F80938000A7
:10029000862D853F58F5193F60F08F5F682E8D17CA
:1002A00008F0612C809181008F5F8F7180938100B5
:1002B0001DC010928100133DA8F0209167002223F9
:1002C00061F06D1202C0612C11C0662019F08150DE
:1002D000682E0CC09150692E09C08F5F682E8D1753
:1002E00090F704C080916300882369F3F7DEEBDEAA
:1002F000062D053F30F4E62DF0E0ED58FF4F00816C
:10030000C02FD0E010E0809181008031A8F1D8DECC
:100310001092810092E6E92E90E0F92EC12CD12CAA
:10032000C1E081E08C0DEFEFCE1ADE0AF70190817B
:100330009F3FB1F06DE570E00ADFF601E559FF4F30
:100340006080F70180818C278083F8DE6FE070E0A9
:1003500080E2FDDEF70180818C278083EFDEB0DE56
:10036000FFEFEF1AFF0A87E0C816D104D1F6612C1F
:1003700000917300C02F74C00E3E81F488E0F82E07
:1003800089E088DE81E290E092DE19BC18BC83E44B
:1003900090E08DDEFA94F110F3CF62C0033F41F498
:1003A00089E078DE8AE090E082DE85E073DE13C0CB
:1003B000043F99F488DE8DDE982F80E0E82FF0E08E
:1003C000E25EFF4FE491E91710F48F5FF7CF6DE71E
:1003D00070E0BDDE75DE74DE43C00E3F81F4612C3B
:1003E00010926900ABDE6AEF70E081E0B0DE81E080
:1003F00080936900A3DE6AEF70E081E0EACF0D3FF1
:1004000091F4612C8FEF80936A0098DE82E042DEE7
:1004100057DE56DE89E03EDEB1DE80936A008EDE76
:100420004FDE4EDEF9CF8C2F8CDEA8DE20916A00E5
:10043000821738F01F5F193078F0C23068F0C15071
:100440000AC090E030E022503109821793071CF473
:10045000C01708F4CF5F10E036DE84EF91E027DEAE
:100460001092810036DE823890F4DF5FD83008F4D5
:100470004ACFCA3020F0D0E0C4E004E044CFC2301C
:1004800040F08C2F86958695C695C80F0C2FD0E02E
:100490003ACF19BC18BC85B7877E806185BFF894B8
:1004A00085B7846885BF8B7F85BF85B7806285BF30
:1004B000889585B78F7D85BFE9CF80E01DDEAECE04
:1004C000E199FECF1FBA8EBBE09A99278DB30895AC
:1004D000262FE199FECF1CBA1FBA8EBB2DBB0FB6DB
:1004E000F894E29AE19A0FBE01960895F894FFCF2E
:00000001FF
